:040000002EEF11F0DE
:1000080000C016F001C015F0E1CF17F0E2CF18F0EC
:100018009DAA66D09EAA64D0AECF56F2ABA20FD0EE
:10002800AB98AECF56F2AB88010E02011C25006ECC
:10003800000E1D21016E00C01CF201C01DF2ABA410
:100048000FD00201AB9EAB8E010E1C25006E000E78
:100058001D21016E00C01CF201C01DF2AECF56F288
:10006800020156510D0A07E05951000802E15851A2
:100078007E0801E314D0010E526F000E536F9D9A53
:100088008F0E5825E16E040E5921E26EE66A58C2B9
:100098008DF459C28EF4586B596B566B21D0595157
:1000A800000802E158517E0805E2020E526F000E68
:1000B800536F9D9A8F0E5825E16E040E5921E26EFA
:1000C80056C2E6FF58C28DF459C28EF4010E582567
:1000D800006E000E5921016E00C058F201C059F29D
:1000E800F2AA0CD0F2A40AD0D76AD66A0001A14BB2
:1000F800A22B010E9F6F000EA06FF2949DA01ED040
:100108009EA01CD002013B4B3C2B0101BD510201BA
:100118003C5D04E10101BC5102013B5D0AE39D9095
:10012800CD903B6B3C6B010E396F000E3A6FCD9052
:100138009D903C0ECF6EB00ECE6E9E9016C000F015
:0E01480015C001F017C0E1FF18C0E2FF110062
:0C01560072B201D0FDD73AC573FF120051
:0E016200ACB202D00000FCD73AC5ADFF1200CF
:10017000C7B409D01F0EC514016E0150000A03E177
:0A018000010E006E01D0006A1200AB
:10018A00F250026EF29E0500FF6A0150FE6E0050A8
:08019A00FD6E02BEF28E1200A0
:0A01A200050E0D6E0D2EFED71200A3
:0A01AC00750E0D6E0D2EFED7120029
:1001B6009E9634C5C9FFD1C035F5D2C036F5D3C039
:1001C60037F5D4C038F5C7A422D00001D151D211D9
:1001D600D311D4111BE005013551361137113811F1
:1001E6000EE145C2E1FF46C2E2FF040EE66E43C2DF
:1001F60000F044C201F0C6DF010E006E3BD0010ED6
:100206000501355F000E365B375B385BDCD7D1C046
:1002160035F5D2C036F5D3C037F5D4C038F59EB61D
:1002260022D00001D151D211D311D4111BE0050106
:1002360035513611371138110EE145C2E1FF46C27C
:10024600E2FF040EE66E43C200F044C201F09ADFFC
:10025600010E006E0FD0010E0501355F000E365BF4
:10026600375B385BDCD7C5BC02D0006A03D0C584D7
:06027600020E006E1200F2
:10027C00D1C036F5D2C037F5D3C038F5D4C039F576
:10028C000501346B356B3551120802E134518E087F
:10029C0008E368DF005201E004D00501344B352B34
:1002AC00F2D70501120E355D02E18F0E345D03E3CA
:1002BC007B0E006E26D0C580C5A022D00001D15186
:1002CC00D211D311D4111BE005013651371138115D
:1002DC0039110EE145C2E1FF46C2E2FF050EE66EA2
:1002EC0043C200F044C201F04ADF010E006E09D097
:1002FC00010E0501365F000E375B385B395BDCD7CE
:04030C00006A120071
:10031000D1C034F5D2C035F5D3C036F5D4C037F5E9
:10032000C582C5A220D00001D151D211D311D41160
:1003300019E0050134513511361137110CE145C270
:10034000E1FF46C2E2FF060EE66E43C200F044C281
:1003500001F01BDF08D0010E0501345F000E355B94
:08036000365B375BDED71200AB
:10036800800E0501356F341F355316E035513415AD
:10037800016E0152010ED8A4000E006E00B002D02A
:100388008B9201D08B8209DF08DF8B840BDF8B9483
:0A03980009DF3533359FE8D7120066
:1003A200000000000000000000000000000000004B
:1003B200000000000000000000000000000000003B
:1003C200000000000000000000000000000000002B
:1003D200000000000000000000000000000000001B
:0403E2000000120005
:1003E600D1C036F5D2C037F5D3C038F5D4C039F50B
:1003F6009E96C5869EB620D00001D151D211D3114A
:10040600D41119E0050136513711381139110CE1B3
:1004160045C2E1FF46C2E2FF030EE66E43C200F0AC
:1004260044C201F0AFDE08D0010E0501365F000EB2
:10043600375B385B395BDED70501C9CF35F53451FB
:10044600000A02E1C58A01D0C59A9E96C588D1C028
:1004560036F5D2C037F5D3C038F5D4C039F59EB6D7
:1004660020D00001D151D211D311D41119E00501C8
:1004760036513711381139110CE145C2E1FF46C238
:10048600E2FF030EE66E43C200F044C201F07ADEDC
:1004960008D0010E0501365F000E375B385B395B0D
:0804A600DED735C500F012009D
:0404AE00C5841200EF
:1004B2008B90060E0C6E300E0D6E0D2EFED70C2E8E
:1004C200FCD700002BC534F54EDF6ADF2CC534F5AE
:1004D2004ADF66DF2BC534F546DF62DF2DC534F512
:1004E20042DF5EDF2BC534F53EDF5ADF2EC534F521
:1004F2003ADF56DF2BC534F536DF52DF2FC534F530
:1005020032DF4EDF2BC534F52EDF4ADF30C534F53E
:100512002ADF46DF2BC534F526DF42DF31C534F54D
:1005220022DF3EDF2BC534F51EDF3ADF32C534F55C
:100532001ADF36DF2BC534F516DF32DF33C534F56B
:1005420012DF2EDF8B801A0E0D6E0D2EFED70000ED
:02055200120095
:1005540005012B51390806E3300E2B5D03E3010E30
:08056400006E01D0006A1200D4
:10056C000450085E0550D8A0053C095E0650D8A082
:10057C00063C0A5E0750D8A0073C0B5E0336070EFC
:10058C000C6E0334083609360A360B36045003A0B9
:10059C000ED0085E0550D8A0053C095E0650D8A0C8
:1005AC00063C0A5E0750D8A0073C0B5E0DD008260F
:1005BC000550D8B0053C09260650D8B0063C0A2692
:1005CC000750D8B0073C0B2603360C2EDAD7023472
:1005DC00083609360A360B36045003A00ED0085ED6
:1005EC000550D8A0053C095E0650D8A0063C0A5E12
:1005FC000750D8A0073C0B5E0DD008260550D8B08C
:10060C00053C09260650D8B0063C0A260750D8B03F
:10061C00073C0B260236070E0C6E023408360936E0
:10062C000A360B36045002A00ED0085E0550D8A036
:10063C00053C095E0650D8A0063C0A5E0750D8A0BF
:10064C00073C0B5E0DD008260550D8B0053C09269A
:10065C000650D8B0063C0A260750D8B0073C0B26EB
:10066C0002360C2EDAD70134083609360A360B3628
:10067C00045002A00ED0085E0550D8A0053C095EBF
:10068C000650D8A0063C0A5E0750D8A0073C0B5E6B
:10069C000DD008260550D8B0053C09260650D8B018
:1006AC00063C0A260750D8B0073C0B260136070E2D
:1006BC000C6E0134083609360A360B36045001A08C
:1006CC000ED0085E0550D8A0053C095E0650D8A097
:1006DC00063C0A5E0750D8A0073C0B5E0DD00826DE
:1006EC000550D8B0053C09260650D8B0063C0A2661
:1006FC000750D8B0073C0B2601360C2EDAD7003445
:10070C00083609360A360B36045001A00ED0085EA6
:10071C000550D8A0053C095E0650D8A0063C0A5EE0
:10072C000750D8A0073C0B5E0DD008260550D8B05A
:10073C00053C09260650D8B0063C0A260750D8B00E
:10074C00073C0B260036070E0C6E003408360936B3
:10075C000A360B36045000A00ED0085E0550D8A007
:10076C00053C095E0650D8A0063C0A5E0750D8A08E
:10077C00073C0B5E0DD008260550D8B0053C092669
:10078C000650D8B0063C0A260750D8B0073C0B26BA
:10079C0000360C2EDAD700B00ED0045008260550C7
:1007AC00D8B0053C09260650D8B0063C0A2607509E
:0807BC00D8B0073C0B26120027
:1007C4000B1E0A1E091E081E082AD8B4092AD8B40A
:0807D4000A2AD8B40B2A120016
:1007DC000B6A0A6A096A00500402F4CF09F0F3CFDD
:1007EC0008F001500502F4CF0BF0F3CF0AF00050E3
:1007FC000502F3500926F4500A22E86A0B22015034
:10080C000402F3500926F4500A22E86A0B2208C0AD
:10081C0000F009C001F00AC002F00BC003F0120096
:10082C0027DDD00E0501346FC0DC2BC534F5BDDCE3
:0A083C002CC534F5BADC35DE1200DD
:10084600086A080E0C6E003408360450085ED8B0EC
:0E08560002D00826D89000360C2EF5D71200DE
:100864002BC500F00032009E0032009E0032009E34
:100874000032009E2CC5E1FF2DC5E2FF300E00249E
:10088400E66E010E05012C25E16E000E2D21E26EAF
:100894000F0E2B15006E300E002600C0E6FF020E70
:0E08A4002C25E16E000E2D21E26EE66A120098
:1008B200E4DCD00E0501346F7DDC2BC534F57ADC27
:1008C20026DDD10E0501346F75DC0501346B8ADD3E
:0C08D20000C034F2EBDD34C200F0120074
:1008DE00020E0C6E080E0D6E0D2EFED70C2EFCD7D2
:0408EE0000001200F4
:1008F2000134083609360450085E0550D8A0053C7C
:10090200095E003601360F0E0C6E013408360936C8
:10091200045000A006D0085E0550D8A0053C095E30
:1009220005D008260550D8B0053C09260036013608
:100932000C2EEBD700B006D0045008260550D8B0D4
:08094200053C0926000012002B
:10094A0025C500F005012507005228E021C5E9FF69
:10095A0022C5EAFFEE50000A0CE021C5E9FF22C5D4
:10096A00EAFF23C5D9FF24C5DAFFEE50DE1801E1FC
:10097A000FD021C5E9FF22C5EAFF23C5D9FF24C547
:10098A00DAFFDE50EE5C006E016A000E015A08D0F2
:10099A000501214B222B234B242BD2D7006A016A53
:0209AA00120039
:1009AC00086A096A100E0C6E0134083609360450B8
:1009BC00085E0550D8A0053C095ED8B007D004509D
:1009CC0008260550D8B0053C0926D89000360136CB
:0609DC000C2EEAD7120008
:1009E2000B0E0C6E570E0D6E0D2EFED70C2EFCD775
:0609F200000000001200ED
:1009F8000450000A12E10550000A0FE10650000AEF
:100A08000CE10750000A09E1FF0E006EFF0E016EAF
:100A1800FF0E026E7F0E036E97D00C6A07BE0C2A7B
:100A28000D6A0B6A0A6A096A086A03500210011003
:100A38000010D8B484D0035007180E6E0EBE0D1ED9
:100A480007AE0BD0041E051E061E071E042AD8B4C6
:100A5800052AD8B4062AD8B4072A03AE0BD0001E3C
:100A6800011E021E031E002AD8B4012AD8B4022A85
:100A7800D8B4032A035007100E6E0EBE1CD072DDC8
:100A88000CBE36D00DAE5BD0001E011E021E031E2A
:100A9800002AD8B4012AD8B4022AD8B4032A081ED6
:100AA800091E0A1E0B1E082AD8B4092AD8B40A2A15
:100AB800D8B40B2A44D007AE15D003BE0DD00350CE
:100AC8000B6E02500A6E0150096E0050086E036AE0
:100AD800026A016A006AD6D7036A026A016A006A72
:100AE800002A000C031E021E011E001E0C8EC7D712
:100AF800082AD8B4092AD8B40A2AD8B40B2A045028
:100B0800085CD8A4BFD70550095CD8A4BBD7065049
:100B18000A5CD8A4B7D707500B5CD8A4B3D70B6A24
:100B28000A6A096A086A002AD8B4012AD8B4022ACB
:100B3800D8B4032A03AEA6D70E6A0E88FF0C0E6A35
:0A0B48000CA001D03BDE000F1200EC
:100B5200220E0C6E086A096A0A6A0B6A0C06D8B47D
:100B62001FD0D8900B320A320932083203320232D5
:100B720001320032D8A0F2D70C06D8B409D0045002
:100B820008260550092206500A2207500B22EAD7EE
:100B9200045008260550092206500A2207500B224B
:020BA20012003F
:100BA4003EEC01F0D00E0501346FDBEC00F00501E2
:100BB400346BDBEC00F088EC01F0D10E0501346FEE
:100BC400DBEC00F0010E0501346F0BDC00C011F505
:100BD400010E0501346F05DC00C010F5010E05019E
:100BE400346FF3EC01F03F0E00140501126F010E97
:100BF400346FF3EC01F0070E0014016E01C014F51C
:100C04000150070802E20501146B0501010E346F5F
:100C1400F3EC01F000C08CF4010E0501346FF3EC29
:100C240001F01F0E001405010F6F346BF3EC01F09B
:100C340000C013F53ADC12C52BF5680E05012C6FC4
:100C4400040E2D6F0DDE3A0E04016A6F10C52BF5EC
:100C54006B0E05012C6F040E2D6F02DE3A0E04019B
:100C64006D6F11C52BF56E0E05012C6F040E2D6FE3
:100C7400F7DD0401706B8CC42BF55A0E05012C6F43
:100C8400020E2D6FEDDD2F0E02015C6F0FC52BF5EB
:100C94005D0E05012C6F020E2D6FE2DD2F0E020199
:100CA4005F6F13C52BF5600E05012C6F020E2D6FBF
:080CB400D7DD0201626B1200A2
:100CBC000201575301E014D005012B6BF4DD7F0EBC
:100CCC0000140401726F736B000E7317000E736FB8
:100CDC0005012B6B72C42CF5A3DD010E0201576FBD
:020CEC001200F4
:100CEE000D0E05013A6FB1EC00F00A0E05013A6FD8
:060CFE00B1EC00F0120051
:100D04000501226B215109081BE20A0E046E21C55C
:100D140000F097DD00C022F500C022F522372291B1
:100D24002237229122372291223722910A0E046E11
:100D340021C500F086DD08C000F00050221302D067
:0A0D440021C522F522C500F01200BF
:100D4E0005012B6BAFDD800E00100401726F736B0B
:100D5E00000E7313000E736F05012B6B72C42CF50E
:080D6E005EDD0201576B12006B
:100D760021C5E9FF22C5EAFFEE500501231905E169
:100D860021C500F022C501F010D021C500F022C512
:100D960001F0214B222B00C0E9FF01C0EAFFEECF94
:0C0DA60000F00052E5E1006A016A120052
:100DB20021C5F6FF22C5F7FF23C5F8FF0900F5CFCD
:100DC20001F00150000812E221C5F6FF22C5F7FF2B
:100DD20023C5F8FF0900F5CF3AF5B1EC00F0010E9A
:0E0DE20005012127000E22232323E2D7120051
:100DF00021C502F022C503F002C000F003C001F0DB
:100E0000024A032A00C0E9FF01C0EAFFEE5201E0F6
:100E1000F3D705012151025C006E22510358016E87
:0A0E2000010E005E000E015A1200E0
:100E2A00030E006E21C528F5000E0501296F00503A
:100E3A0005E0283728912937FF0FFAD72A6B3E0E8B
:100E4A002125F66E3D0EF76E000EF722000EF86EA3
:100E5A00000EF8220900F5CF68F2266B276B800E88
:100E6A002719006E800E005C02E1080E265DD8B0DC
:100E7A00D6D0400E246F000E256F800E006E800EB5
:100E8A002519005C02E12451000819E2680E2425A4
:100E9A00E16E020E2521E26E010E245D006E000E47
:100EAA002559016E680E0024E96E020E0120EA6ED1
:100EBA00EECFE6FF010E245F000E255BDED7285138
:100ECA002625006E29512721016E3E0E0024F66E5A
:100EDA003D0E0120F76E000EF86E000E01BEFF0EE9
:100EEA00F8220900F5CF68F22A6B080E246F000E6B
:100EFA00256F800E006E800E2519005C02E12451D8
:100F0A00000876E224C52BF5680EE96E020EEA6E39
:100F1A002A51E926D8B0EA2AEECF2CF5080E2A255E
:100F2A00006E016A000E0122680E0024E96E020EAC
:100F3A000120EA6EEECF2DF5100E2A25006E016A09
:100F4A00000E0122680E0024E96E020E0120EA6EEC
:100F5A00EECF2EF5180E2A25006E016A000E012228
:100F6A00680E0024E96E020E0120EA6EEECF2FF51C
:100F7A00200E2A25006E016A000E0122680E002446
:100F8A00E96E020E0120EA6EEECF30F5280E2A2510
:100F9A00006E016A000E0122680E0024E96E020E3C
:100FAA000120EA6EEECF31F5300E2A25006E016A75
:100FBA00000E0122680E0024E96E020E0120EA6E7C
:100FCA00EECF32F5380E2A25006E016A000E012294
:100FDA00680E0024E96E020E0120EA6EEECF33F5A8
:100FEA0059EC02F02A2B010E245F000E255B81D7F3
:100FFA00246B256B2351255D02E12251245D0CE20D
:10100A00150E0C6EC60E0D6E0D2EFED70C2EFCD7CD
:10101A000000244B252BEED7264B272B20D7120076
:10102A00A69C22C5AAFF21C5A9FFA69EA680A8CF75
:04103A0000F01200B0
:10103E00020E0C6E9D0E0D6E0D2EFED70C2EFCD7D5
:06104E000000000012008A
:1010540021C5E9FF22C5EAFFEECF23F5000E050105
:10106400246F000E246F000E241902E1200E2319B0
:1010740007E0000E241902E1090E231901E003D050
:10108400214B222BE5D7256B266B276B286B000E93
:10109400241902E12D0E231905E1274B282B214B9E
:1010A400222B08D0000E241902E12B0E231902E191
:1010B400214B222B21C5E9FF22C5EAFFEECF23F500
:1010C400000E246F000E246F23C52BF5AAEC02F04A
:1010D400005219E025C500F026C501F00A0E046E81
:1010E400000E056EEEEC03F0300E235D026E000E72
:1010F4002459036E02500024256F03500120266FEB
:10110400214B222BD7D72751281108E0255100085D
:10111400006E26C501F0000E015604D025C500F06E
:0611240026C501F01200D7
:10112A00090E0B6E1E0E0C6EE40E0D6E0D2EFED702
:0C113A000C2EFCD70B2EFAD70000120080
:1011460019C501F0010E006E015004E00036009052
:10115600FF0FFBD700C01DF5001E00C01CF517C50C
:10116600E9FF18C5EAFF0050EF16120EE926050141
:101176001B6B1B51070815E31BC500F01AC501F0D0
:10118600005004E00132019EFF0FFBD71C51EF1601
:1011960001A002D01D51EF124FDF1D51EF121B2B84
:1011A600E8D7120EE95E6FEC04F06FEC04F0120063
:1011B600060E0C6E300E0D6E0D2EFED70C2EFCD7C5
:0411C6000000120013
:1011CA0019C501F0010E006E015004E000360090CE
:1011DA00FF0FFBD700C01BF5001E17C5E9FF18C596
:1011EA00EAFF0050EF16120EE9260050EF16F1EC56
:1011FA0004F005011B51EF12120EE95E1BDF1B51B1
:10120A00EF141A6F1A51000A000ED8A4010E1A6FB1
:0A121A00F1EC04F01AC500F0120018
:1012240019C504F01AC505F017C502F018C503F076
:101234001BC500F01CC501F0010E05011B5F000E6B
:101244001C5B005001100FE004C0E9FF05C0EAFF79
:1012540002C0E1FF03C0E2FFEECFE6FF024A032A29
:10126400044A052AE5D717C500F018C501F0120095
:1012740005011A6B17C5E9FF18C5EAFFEECF19F58A
:101284001951000A0FE019C53AF5B1EC00F0050157
:101294001A2B1A511725E96E000E1821EA6EEECFAB
:0612A40019F5EED712005F
:1012AA0019C5F6FF1AC5F7FF1BC5F8FF0900F5CFE8
:1012BA0000F0005218E019C5F6FF1AC5F7FF1BC562
:1012CA00F8FF0900F5CF00F017C5E1FF18C5E2FFE6
:1012DA0000C0E6FF0501174B182B010E1927000E57
:1012EA001A231B23DDD717C5E1FF18C5E2FFE66AFB
:0212FA001200E0
:1012FC0005011B6B050E1B5D0AE21B511925E16EE6
:10130C00000E1A21E26E200EE66E1B2BF3D71B513A
:10131C001925E16E000E1A21E26EE66A1B071B51BD
:10132C0019251C6F000E1A211D6F0A0E046E000E7B
:10133C00056E17C500F018C501F0D6EC04F008C016
:10134C0000F009C001F0300E00261CC5E1FF1DC5E0
:10135C00E2FF00C0E6FF0A0E046E000E056E17C514
:10136C0000F018C501F0D6EC04F000C017F501C070
:10137C0018F5000E011802E1000E001801E102D070
:06138C001B07CDD7120083
:1013920017C51BF518C51CF51BC521F51CC522F583
:1013A20043DE00C01DF50050000A01E12FD0800E7F
:1013B200006E800E05011C19005C02E11B51FE0843
:1013C20001E224D01DC53AF5B1EC00F00501175138
:1013D2001B5D006E18511C59016E00501925E16EFB
:1013E20001501A21E26E1DC5E6FF030E0B6E080EB8
:1013F2000C6E770E0D6E0D2EFED70C2EFCD70B2E1B
:0E140200FAD71B4B1C2B1D51000AC6E112002D
:10141000130E806E0F01386B0F0E926E92988988B2
:1014200092869280FF0E816E396BFF0E936E9382CF
:10143000826AFF0E946E3A6B948E948C9490949280
:1014400094948B80D1EC01F08B92D1EC01F08B94D1
:0A145000D1EC01F0C56A60941200AF
:10145A000900F5CFE6FF0006FBE10106F9E11200FB
:10146A003B0E0501216F4D0E226F000E236F9CDC8F
:10147A00290E0B6E960E0C6E7F0E0D6E0D2EFED77C
:10148A000C2EFCD70B2EFAD7430E0501216F4C0EFA
:10149A00226F000E236F88DC290E0B6E960E0C6EDF
:1014AA007F0E0D6E0D2EFED70C2EFCD70B2EFAD703
:1014BA00360E0501216F4C0E226F000E236F74DC6D
:1014CA00290E0B6E960E0C6E7F0E0D6E0D2EFED72C
:1014DA000C2EFCD70B2EFAD79F0E0501216F4B0E4F
:1014EA00226F000E236F60DC290E0B6E960E0C6EB7
:1014FA007F0E0D6E0D2EFED70C2EFCD70B2EFAD7B3
:10150A00760E0501216F4B0E226F000E236F4CDC05
:10151A00290E0B6E960E0C6E7F0E0D6E0D2EFED7DB
:10152A000C2EFCD70B2EFAD7680E0501216F4C0E34
:10153A00226F000E236F38DC290E0B6E960E0C6E8E
:10154A007F0E0D6E0D2EFED70C2EFCD70B2EFAD762
:10155A00740E0501216F4C0E226F000E236F24DCDE
:10156A00290E0B6E960E0C6E7F0E0D6E0D2EFED78B
:0A157A000C2EFCD70B2EFAD712003E
:10158400620E02012A6F010E2B6F3A0E2C6F050EAC
:101594002D6FFF0E186FFF0E196F000E1A6F000EDD
:1015A4001B6FFF0E146FFF0E156F000E166F000EEB
:1015B400176FFF0E1E6FFF0E1F6F000E206F000EC1
:1015C400216FAC8A900EAB6E948E949C9EAA03D02D
:0815D400AECF00F0FBD71200BE
:1015DC00050118AF0FD02D0E00019E6F19C5E1FF4C
:1015EC001AC5E2FF2D0EE66E0501171F181F174BCB
:1015FC00182B09D02B0E00019E6F19C5E1FF1AC5DF
:10160C00E2FF200EE66E17C500F018C501F001329E
:10161C000032019E01320032019E01320032019EE5
:10162C0001320032019E00C032F201C033F2010ED1
:10163C00050119251B6F000E1A211C6F0A0E046E72
:10164C00000E056ED6EC04F00A0E046E000E056E4C
:10165C00D6EC04F008C000F009C001F0300E0026F2
:10166C001BC5E1FF1CC5E2FF00C0E6FF020E1925F9
:10167C001B6F000E1A211C6F0A0E046E000E056EF5
:10168C0032C200F033C201F0D6EC04F008C000F016
:10169C0009C001F0300E00261BC5E1FF1CC5E2FF9E
:1016AC0000C0E6FF17C535F218C536F2000E020170
:1016BC00376F386F0F0E3517000E36173717381770
:1016CC00080E05011925E16E000E1A21E26EE66A7C
:1016DC0035C200F036C201F037C202F038C203F056
:1016EC00710E046E020E056E000E066E076EA9ECEE
:1016FC0005F000C035F201C036F202C037F203C06B
:10170C0038F2030E1925E16E000E1A21E26E2E0E30
:10171C00E66E040E19251B6F000E1A211C6FE80EC5
:10172C00046E030E056E000E066E076E35C200F0D9
:10173C0036C201F037C202F038C203F0FCEC04F000
:10174C00300E00261BC5E1FF1CC5E2FF00C0E6FF02
:10175C00050E050119251B6F000E1A211C6F640E56
:10176C00046E000E056E066E076E35C200F036C2B2
:10177C0001F037C202F038C203F0FCEC04F00A0EA0
:10178C00046E000E056E066E076EFCEC04F008C0CD
:10179C0000F009C001F00AC002F00BC003F0300EDB
:1017AC0000261BC5E1FF1CC5E2FF00C0E6FF060ECC
:1017BC0005011925E16E000E1A21E26EE66A32C2AD
:1017CC0000F033C201F0000E026E036EE80E046EE0
:1017DC00030E056E000E066E000E076EA9EC05F0EA
:1017EC0000C01BF501C01CF502C01DF503C01EF5A1
:1017FC000A0E046E000E056E066E076E35C200F002
:10180C0036C201F037C202F038C203F0FCEC04F02F
:10181C00005005011B250001D56F015005011C214D
:10182C000001D66F025005011D210001D76F035036
:10183C0005011E210001D86F9E512D0A14E1006A8A
:10184C00016A026A036AD551005ED651015AD7511A
:10185C00025AD851035A00C0D5F001C0D6F002C0CC
:0C186C00D7F003C0D8F09EC000F01200BE
:10187800000E0501181902E1000E171937E017C507
:10188800E9FF18C5EAFFEE5231E019C521F51AC57E
:1018980022F5F8EC06F000C025F517C521F518C5A6
:1018A80022F519C523F51AC524F5A5EC04F0000E98
:1018B800011802E1000E001805E117C500F018C56F
:1018C80001F016D0010E05011725216F000E182111
:1018D800226F19C5E9FF1AC5EAFFEECF23F5BBEC65
:1018E80006F000C017F501C018F5C2D7006A016AF2
:0218F8001200DC
:1018FA0017C504F018C505F004C002F005C003F0CE
:10190A00044A052A19C500F01AC501F00501194B48
:10191A001A2B00C0E9FF01C0EAFF02C0E1FF03C0C1
:10192A00E2FFEECFE6FF02C0E9FF03C0EAFFEE5294
:0E193A0001E0E2D717C500F018C501F0120059
:1019480017C504F018C505F004C0E9FF05C0EAFF93
:10195800EE5203E0044A052AF7D704C002F005C096
:1019680003F0044A052A19C500F01AC501F005015B
:10197800194B1A2B00C0E9FF01C0EAFF02C0E1FFC2
:1019880003C0E2FFEECFE6FF02C0E9FF03C0EAFFB3
:10199800EE5201E0E2D717C500F018C501F01200B9
:1019A8000450000A08E10550000A05E1FF0E006E28
:1019B8007F0E016E58D00D6A096A086A015000103E
:1019C800D8B4000C015005180A6E0ABE0D1E0B6A29
:1019D80005AE05D0041E051E042AD8B4052A01AE9A
:1019E80005D0001E011E002AD8B4012A0150051096
:1019F8000A6E0ABE10D079EC04F00BB020D00DAE00
:101A0800000C001E011E002AD8B4012A081E091E57
:101A1800082AD8B4092A000C05AE0DD001BE07D09B
:101A28000150096E0050086E016A006AE8D7016A21
:101A3800006A002A000C011E001E0B2ADDD7082AA6
:101A4800D8B4092A0450085CD8A4D9D70550095C31
:101A5800D8A4D5D7096A086A002AD8B4012A01AEE1
:081A6800CED70000FF0C1200B4
:101A700005011B6B1C6B19511B25216F1A511C2171
:101A8000226F15EC08F000C01DF50050000A01E1BE
:101A900020D0800E006E800E1C19005C02E11B51EC
:101AA0001F0801E216D01B511725E16E1C511821A9
:101AB000E26E1DC5E6FF150E0C6EC60E0D6E0D2EE8
:101AC000FED70C2EFCD700001B4B1C2B1D51000A0F
:101AD000D2E11B511725006E1C511821016E010E19
:0E1AE000005CE16E000E0158E26EE66A120034
:101AEE00020E0501176F000E186F77EC06F0050158
:101AFE001B6B1C6B9D9A8F0E04018D25E16E040EDF
:101B0E008E21E26EE66A800E8E19006E800E005CEB
:101B1E0002E1160E8D5DD8B0EAD0800E006E800EFA
:101B2E008E19005C02E18D511308D8B0E0D0020E80
:101B3E000501196F000E1A6F800E1A19006E800EB5
:101B4E0004018E19005C03E18D510501195D32E22D
:101B5E0005018F0E1925E96E040E1A21EA6EEECFDD
:101B6E0001F001503B0A23E18F0E1925E16E040EA0
:101B7E001A21E26EE66A740E1B251F6F040E1C21DD
:101B8E00206F8F0E1725216F040E1821226F2AEC5D
:101B9E0008F01FC5E1FF20C5E2FF00C0E6FF1B4BAA
:101BAE001C2B010E1925176F000E1A21186F194BD9
:101BBE001A2BC2D70501740E1B251F6F040E1C2194
:101BCE00206F8F0E1725216F040E1821226F2AEC1D
:101BDE0008F01FC5E1FF20C5E2FF00C0E6FF79C493
:101BEE001DF5000E1E6F78C479F477C478F41DC508
:101BFE0077F474C48CF475C40FF576C413F51DC553
:101C0E0014F51D5107080AE2070E146F630E216FBB
:101C1E004A0E226F000E236FD9EC06F078C412F52F
:101C2E0079C410F50501116BA7EC06F005012B6BBD
:101C3E002C6B16EC04F010C521F582EC06F000C0FA
:101C4E002CF5010E2B6F16EC04F012C521F582EC6B
:101C5E0006F000C02CF5020E2B6F16EC04F014C526
:101C6E0021F582EC06F000C02CF5030E2B6F16EC5E
:101C7E0004F08CC421F582EC06F000C02CF5040EA5
:101C8E002B6F16EC04F00FC521F582EC06F000C0A8
:101C9E002CF5050E2B6F16EC04F013C521F582EC16
:101CAE0006F000C02CF5060E2B6F16EC04F0070E96
:101CBE0005012B6F100E2C6F16EC04F0E30E0501D0
:101CCE00216F4A0E226F000E236FD9EC06F077ECCF
:101CDE0006F0C50E0501216F4B0E226F000E236F0D
:101CEE00D9EC06F05EEC06F0D2EC05F012D0C00E88
:101CFE000501216F470E226F000E236FD9EC06F0FF
:101D0E00950E0501216F460E226F000E236FD9EC42
:041D1E0006F01200B9
:101D2200A6A202D00000FCD7A69C18C5AAFF17C520
:101D3200A9FF19C5A8FFA69EA684F2CF00F0F29EC5
:101D4200550EA76EAA0EA76EA68200BE02D0F29E04
:101D520001D0F28EA694A1B802D00000FCD7A198BF
:021D620012006D
:101D640018C500F00032009E0032009E0032009E32
:101D74000032009EF90E0024F66E4B0EF76E000E34
:101D8400F722000EF86E000EF8220900F5CF00F0DD
:101D940019C5E1FF1AC5E2FF00C0E6FF010E050107
:101DA4001925E16E000E1A21E26E0F0E1815006E51
:101DB400F90E0024F66E4B0EF76E000EF722000E9D
:101DC400F86E000EF8220900F5CF00F000C0E6FF1F
:101DD400020E1925E16E000E1A21E26E17C500F0FD
:101DE4000032009E0032009E0032009E0032009EAF
:101DF400F90E0024F66E4B0EF76E000EF722000E5D
:101E0400F86E000EF8220900F5CF00F000C0E6FFDE
:101E1400030E1925E16E000E1A21E26E0F0E17153E
:101E2400006EF90E0024F66E4B0EF76E000EF722CC
:101E3400000EF86E000EF8220900F5CF00F000C085
:101E4400E6FF040E1925E16E000E1A21E26EE66A21
:021E540012007A
:101E560005011A6B030E1A5D0AE21A511825E16E86
:101E6600000E1921E26E200EE66E1A2BF3D71A51D8
:101E76001825E16E000E1921E26EE66A1A071A515C
:101E860018251B6F000E19211C6F0A0E046E17C54C
:101E960000F023EC04F008C000F0300E00261BC54D
:101EA600E1FF1CC5E2FF00C0E6FF0A0E046E17C57F
:101EB60000F023EC04F000C017F50050000A01E121
:081EC60002D01A07DCD712005C
:0E1ECE00948A94929494829A8B928B94120030
:101EDC000501176B186B8B80090E0B6E1E0E0C6EAA
:101EEC00E40E0D6E0D2EFED70C2EFCD70B2EFAD752
:101EFC0000008B900C0E2B6F010E2C6F010E2D6FB2
:101F0C00010E2E6F010E2F6F010E306F010E316F0F
:101F1C00010E326F010E336F59EC02F0090E2B6F6C
:101F2C002C6B2D6B2E6B2F6B306B316B326B336BD1
:101F3C0059EC02F00B0E2B6F070E2C6F070E2D6F4A
:101F4C00070E2E6F070E2F6F070E306F070E316FB7
:101F5C00070E326F070E336F59EC02F00F0E2B6F1A
:101F6C002C6B2D6B2E6B2F6B306B316B326B336B91
:101F7C0059EC02F00A0E2B6F2C6B2D6B2E6B2F6B0A
:101F8C00306B316B326B336B59EC02F0176B186B97
:101F9C00800E1819006E800E005C02E1080E175DB1
:101FAC0010E21751010F2B6F2C6B2D6B2E6B2F6BBF
:101FBC00306B316B326B336B59EC02F0174B182BC7
:101FCC00E7D78B80D00E0C6EC90E0D6E0D2EFED782
:0A1FDC000C2EFCD7000000001200DC
:101FE60019C501F0010E006E015004E000360090A4
:101FF600FF0FFBD700C01DF5001C05011C6F1B6BF6
:1020060017C5E9FF18C5EAFF1A6B1A51070824E33A
:102016001C51EF16120EE9261C51EF16D1EC00F0FA
:102026001D51EF12D1EC00F0120EE95E1D51EF14B6
:10203600006E0CE01AC501F0010E006E015004E0BE
:1020460000360090FF0FFBD700501B136FEC04F017
:0E2056006FEC04F01A2BD9D71BC500F0120056
:1020640017C500F00032009E0032009E0032009E30
:102074000032009EF90E0024F66E4B0EF76E000E31
:10208400F722000EF86E000EF8220900F5CF00F0DA
:1020940018C5E1FF19C5E2FF00C0E6FF010E050106
:1020A4001825E16E000E1921E26E0F0E1715006E51
:1020B400F90E0024F66E4B0EF76E000EF722000E9A
:1020C400F86E000EF8220900F5CF00F000C0E6FF1C
:1020D400020E1825E16E000E1921E26EE66A120066
:1020E4000501176B186B800E1819006E800E005CCA
:1020F40002E1080E175D10E21751010F2B6F2C6BD4
:102104002D6B2E6B2F6B306B316B326B336B59EC49
:0A21140002F0174B182BE7D712005A
:10211E0017C5E9FF18C5EAFFEE5000080FE217C514
:10212E00E9FF18C5EAFFEECF21F519C522F51AC54C
:0E213E0023F515EC07F0174B182BEAD712000B
:10214C000201586B596B000E595D02E1800E585D0F
:10215C0012E28F0E5825E16E040E5921E26EE66AEA
:10216C00010E5825006E000E5921016E00C058F268
:10217C0001C059F2E8D7586B596B04018D6B8E6B0B
:10218C00AECF56F20201566B526B536B9D8A546B59
:04219C00556B12006D
:1021A000700E02013F6F010E406F000E416F000E76
:1021B000426F7C0E4B6F020E4C6F000E4D6F000E87
:1021C0004E6F100E476F030E486F000E496F000EE2
:1021D0004A6FE60E266F030E276F340E286F050E2A
:1021E000296FB60E226F010E236F340E246F050E79
:1021F000256FAE0E2E6F040E2F6F000E306F000E87
:10220000316F949894968B988B9694889486C79EF9
:08221000C79C380EC66E1200D7
:1022180017C5F6FF18C5F7FF19C5F8FF0900F5CF70
:1022280001F00150000815E217C5F6FF18C5F7FFC1
:1022380019C5F8FF0900F5CF21F51AC522F51BC508
:1022480023F515EC07F0010E1727000E18231923A4
:04225800DFD71200BA
:10225C00A4EC26F0D38CD38AD3889B8CD392D390C6
:10226C0008EC0AF0520E0B6E2B0E0C6E000E0D6E5F
:10227C000D2EFED70C2EFCD70B2EFAD7000000002B
:10228C00F282D384F28EF28C030E8A6E00008B8065
:10229C00520E0B6E2B0E0C6E000E0D6E0D2EFED70D
:1022AC000C2EFCD70B2EFAD70000100E0101BC6FC0
:1022BC00000EBD6F8998B886030EB06E400EAF6EDF
:1022CC00AC84C2EC0AF0090E0B6E1E0E0C6EE40E02
:1022DC000D6E0D2EFED70C2EFCD70B2EFAD7000050
:1022EC000C0E05013A6FB1EC00F0290E0B6E960E38
:1022FC000C6E7F0E0D6E0D2EFED70C2EFCD70B2EFA
:10230C00FAD7E80E0101BA6F000EBB6F6A0E00011E
:10231C00E66F010EE76FE86B01016A6B3E0E05017B
:10232C00216F490E226F000E236FD9EC06F035ECAD
:10233C000AF0520E0B6E2B0E0C6E000E0D6E0D2E47
:10234C00FED70C2EFCD70B2EFAD7000077EC06F03C
:10235C00E80E0501216F4B0E226F000E236FD9EC96
:10236C0006F00101686B696B800E6919006E800EB6
:10237C00005C02E10B0E685D29E2030E006E000E9C
:10238C00016E68C104F069C105F0EEEC03F0670E54
:10239C000024E96E000E0120EA6EEECF21F5EECF9F
:1023AC0022F5EECF23F5D9EC06F0090E0B6E1E0EBE
:1023BC000C6EE40E0D6E0D2EFED70C2EFCD70B2ED4
:1023CC00FAD700000101684B692BCED7520E0B6E69
:1023DC002B0E0C6E000E0D6E0D2EFED70C2EFCD798
:1023EC000B2EFAD7000077EC06F077EC06F0000E17
:1023FC000101C26FFA0EC36FBAC117F5BBC118F554
:10240C00B30E0501196F490E1A6F000E1B6F55ECB8
:10241C0009F0C2C117F5C3C118F5C40E0501196F37
:10242C00010E1A6F7EEC09F0170E0101BA25050199
:10243C00176F000E0101BB210501186FC40E196F37
:10244C00010E1A6F050E1B6F000E1C6F12EC09F0BB
:10245C00BAC117F5BBC118F53AEC09F08E0E216F15
:10246C00490E226F000E236FD9EC06F0E80E010125
:10247C00BA6F000EBB6F0501176B186BBAC119F55B
:10248C00BBC11AF5C9EC09F077EC06F0030E0B6E24
:10249C00080E0C6E770E0D6E0D2EFED70C2EFCD783
:1024AC000B2EFAD7060E0101BA25E96E000EBB21E0
:1024BC00EA6E300EEE5C006E0A0E0002F3CF01F0F5
:1024CC0001C094F0070EBA25E96E000EBB21EA6E2E
:1024DC00300EEE5C006E0050012601C094F0020E2E
:1024EC00015C05E300019451620801E303D0000193
:1024FC00140E946F100E0501176F000E186FBAC1F1
:10250C0019F5BBC11AF5C9EC09F077EC06F0020E0F
:10251C000B6EA00E0C6E920E0D6E0D2EFED70C2EA9
:10252C00FCD70B2EFAD70000040E0101BA25E96E78
:10253C00000EBB21EA6E300EEE5C0001606F0A0EDD
:10254C006003F3CF60F0050E0101BA25E96E000EB1
:10255C00BB21EA6E300EEE5C006E0050000160276D
:10256C00200E0501176F000E186FBAC119F5BBC10B
:10257C001AF5C9EC09F077EC06F0030E0B6E080E99
:10258C000C6E770E0D6E0D2EFED70C2EFCD70B2E6F
:10259C00FAD7060E0101BA25E16E000EBB21E26EE0
:1025AC00E66A040EBA250501216F000E0101BB215C
:1025BC000501226F2AEC08F000C0BEF1090E0101E2
:1025CC00BA25E16E000EBB21E26EE66A070EBA2553
:1025DC000501216F000E0101BB210501226F2AECC0
:1025EC0008F000C0C1F10101C08160C034F0336A51
:1025FC00400E0501176F000E186FBAC119F5BBC15B
:10260C001AF5C9EC09F077EC06F0020E0B6EA00E71
:10261C000C6E920E0D6E0D2EFED70C2EFCD70B2EC3
:10262C00FAD70000040E0101BA25E96E000EBB2199
:10263C00EA6E300EEE5C356E0A0E3502F3CF35F0D5
:10264C00050EBA25E96E000EBB21EA6E300EEE5C6B
:10265C00006E0050352677EC06F08B0E0501216FCD
:10266C004B0E226F000E236FD9EC06F095EC08F0A0
:10267C000001E26BE36B800E0501176F0F0E186FF4
:10268C00196BE5EC08F0DBEC08F0800E176F0F0E01
:10269C00186F196B330E1A6FA3EC08F0DBEC08F013
:1026AC00800E176F0F0E186F196B97DC00C056F267
:1026BC00DBEC08F0190E216F4C0E226F000E236F0D
:1026CC00D9EC06F00101C46B56C217F5C40E050116
:1026DC00186F010E196FC0DCC40E176F010E186F46
:1026EC003AEC09F0FB0E216F4C0E226F000E236F9B
:1026FC00D9EC06F00101686B696B800E6919006EEC
:10270C00800E005C02E1060E685D27E2800E05017A
:10271C00176F0F0E186F196B60DC00C056F2DBECF4
:10272C0008F0D90E01016825E16E000E6921E26EF8
:10273C0056C2E6FFC46B56C217F5C40E0501186FDE
:10274C00010E196F89DCC40E176F010E186F3AEC6D
:10275C0009F00101684B692BD0D7E30E0501216FFD
:10276C004C0E226F000E236FD9EC06F0800E050183
:10277C00176F0F0E186F196B30DC00C056F2010189
:10278C00C46B56C217F5C40E0501186F010E196FF4
:10279C0063DCC40E176F010E186F3AEC09F077EC7E
:1027AC0006F0880E0501216F470E226F000E236F75
:1027BC00D9EC06F067EC0FF0090E0B6E1E0E0C6ECA
:1027CC00E40E0D6E0D2EFED70C2EFCD70B2EFAD769
:1027DC0000006EEC0FF0020E216F4B0E226F000EFC
:1027EC00236FD9EC06F078DC520E0B6E2B0E0C6EB0
:1027FC00000E0D6E0D2EFED70C2EFCD70B2EFAD71D
:10280C000000A00EC86EC6DC150E0501216F470E28
:10281C00226F000E236FD9EC06F0090E0B6E1E0E04
:10282C000C6EE40E0D6E0D2EFED70C2EFCD70B2E5F
:10283C00FAD70000D70E0501216F4B0E226F000E48
:10284C00236FD9EC06F077EC06F0D2EC05F0090E0C
:10285C000501216F4C0E226F000E236FD9EC06F090
:10286C00030E006E000E016E14C504F0000E056E12
:10287C00EEEC03F0190E0024E96E000E0120EA6E56
:10288C00EECF21F5EECF22F5EECF23F5D9EC06F005
:10289C00200E05013A6FB1EC00F05A0E0501176FCE
:1028AC00020E186F3AEC09F0DB0E216F4C0E226F02
:1028BC00000E236FD9EC06F0680E0501176F040E9D
:1028CC00186F3AEC09F077EC06F0F28CD08EF28CA3
:1028DC00F28E280E0101BC6F000EBD6F77EC06F076
:1028EC0072EC10F0130E216F490E226F000E236F45
:1028FC00D9EC06F01A0E0501216F4B0E226F000E5B
:10290C00236FD9EC06F00101686B696B0A0E0501A7
:10291C002B6F2C6B2D6B2E6B2F6B306B316B326BDB
:10292C00336B59EC02F0AE0E176F4C0E186F000E95
:10293C00196F140E1A6F000E1B6F68DC9C0E0501CC
:10294C00176F4C0E186F000E196F280E1A6F000EB1
:10295C001B6F5CDC8978520E0B6E2B0E0C6E000E0E
:10296C000D6E0D2EFED70C2EFCD70B2EFAD70000B9
:10297C007B0E0501216F450E226F000E236FD9ECE3
:10298C0006F00A0E05012B6F0F0E2C6F0D0E2D6F1E
:10299C000A0E2E6F080E2F6F060E306F030E316F5E
:1029AC00020E326F336B59EC02F0F40E0B6E820E8A
:1029BC000C6E050E0D6E0D2EFED70C2EFCD70B2EAD
:1029CC00FAD7B90E216F480E226F000E236FD9EC87
:1029DC0006F035C068F1000E0101696F0A0E0501A1
:1029EC002B6F68C12CF568C12DF568C12EF568C137
:1029FC002FF568C130F568C131F568C132F568C191
:102A0C0033F559EC02F0520E0B6E2B0E0C6E000EC1
:102A1C000D6E0D2EFED70C2EFCD70B2EFAD7000008
:102A2C0072EC10F0C90E176F4C0E186F000E196F68
:102A3C000A0E1A6F000E1B6F0CEC11F0E80E010160
:102A4C00BA6F000EBB6FBF8B0001E16B0001F29EF1
:102A5C00030EE115016E0150000A3BE16EEC0FF024
:102A6C0072EC10F0E80E0101BA6F000EBB6FBAC128
:102A7C0017F5BBC118F5D20E0501196F4C0E1A6F64
:102A8C00000E1B6F55EC09F0BAC117F5BBC118F558
:102A9C00010E0501196F000E1A6F8FEC10F0010179
:102AAC00686B696B800E6919006E800E005C02E128
:102ABC00500E685D0AE26851BA25E16E6951BB217E
:102ACC00E26EE66A684B692BEDD7E80EBA6F000E22
:102ADC00BB6FA6EC10F0F28E520E0B6E2B0E0C6E22
:102AEC00000E0D6E0D2EFED70C2EFCD70B2EFAD72A
:102AFC000000E80E0101BA6F000EBB6F090E050154
:102B0C00216F4D0E226F000E236FD9EC06F0E1C041
:102B1C0017F5C40E0501186F010E196F2BEC0FF091
:102B2C00C40E176F010E186F3AEC09F0200E3A6FB5
:102B3C00B1EC00F06A0E0001E66F010EE76FE80ED3
:102B4C000101BA6F000EBB6F800E0501176F0F0EDF
:102B5C00186F196BE5EC08F0800E176F0F0E186FDD
:102B6C00196BCC0E1A6FA3EC08F0800E176F0F0EBA
:102B7C00186F196B440E1A6FA3EC08F0DBEC08F01D
:102B8C00800E176F0F0E186F196BE5EC08F0800EA6
:102B9C00176F0F0E186F196BCC0E1A6FA3EC08F091
:102BAC00800E176F0F0E186F196BBE0E1A6FA3ECF9
:102BBC0008F0800E176F0F0E186F196BF3EC0FF0F7
:102BCC0000C031F0000E326E800E176F0F0E186FB2
:102BDC00196BF3EC0FF000C062F00001616B315027
:102BEC00612732506223D2EC05F03B0E05013A6F9F
:102BFC00B1EC00F0030E006E000E016E14C504F073
:102C0C00000E056EEEEC03F0190E0024E96E000EBA
:102C1C000120EA6EEECF21F5EECF22F5EECF23F5B3
:102C2C00D9EC06F03B0E05013A6FB1EC00F05A0EF0
:102C3C000501176F020E186F3AEC09F03B0E3A6F54
:102C4C00B1EC00F0680E0501176F040E186F3AEC2A
:102C5C0009F03B0E3A6FB1EC00F0E6C021F5E7C08D
:102C6C0022F5F8EC06F0800E026E800E0118025C64
:102C7C0002E1005007081CE20101C0A103D060C0B2
:102C8C0034F0C091345000080DE2E6C017F5E7C0EF
:102C9C0018F594C019F5000E05011A6F8FEC10F0A1
:102CAC00340605D0E6C0E1FFE7C0E2FFE66A08D1D2
:102CBC00280E0101BC6F000EBD6FE80EBA6F000E3E
:102CCC00BB6FC40E0501176F010E186F030E006E5B
:102CDC00000E016E14C504F0000E056EEEEC03F050
:102CEC00190E0024E96E000E0120EA6EEECF19F5E4
:102CFC00EECF1AF5EECF1BF555EC09F0BAC117F56E
:102D0C00BBC118F5C40E0501196F010E1A6F7DECCD
:102D1C000CF0BAC121F5BBC122F5F8EC06F000C0ED
:102D2C00E4F001C0E5F000500101BA250501176F70
:102D3C0001500101BB210501186F650E196F000EC2
:102D4C001A6FA4EC0CF0BAC117F5BBC118F55A0EEA
:102D5C00196F020E1A6FA4EC0CF0BAC121F5BBC1AD
:102D6C0022F5F8EC06F000C0E4F001C0E5F00050EC
:102D7C000101BA250501176F01500101BB210501A5
:102D8C00186F630E196F000E1A6FA4EC0CF0BAC119
:102D9C0021F5BBC122F5F8EC06F000C0E4F001C04F
:102DAC00E5F000500101BA250501176F0150010132
:102DBC00BB210501186F680E196F040E1A6FA4EC75
:102DCC000CF061C017F562C018F5C40E196F010E36
:102DDC001A6FEEEC0AF0C40E0501216F010E226F82
:102DEC00F8EC06F000C0E4F001C0E5F0C40E0024DD
:102DFC00176F010E0120186F400E196F4D0E1A6FD0
:102E0C00000E1B6F55EC09F0C40E0501176F010E77
:102E1C00186F3AEC09F077EC06F0C40E0501216F3F
:102E2C00010E226FF8EC06F000C0E4F001C0E5F0F2
:102E3C000101686B696B800E6919006E800E0001D0
:102E4C00E519005C03E1E4510101685D15E2010143
:102E5C00C40E6825E96E010E6921EA6EEE50B00AC7
:102E6C0008E1C40E6825E16E010E6921E26E7E0E4A
:102E7C00E66E684B692BDFD7BAC121F5BBC122F5D1
:102E8C00F8EC06F000C0E4F001C0E5F000500101E0
:102E9C00BA250501176F01500101BB210501186FFF
:102EAC00C40E196F010E1A6FA4EC0CF0BAC117F511
:102EBC00BBC118F594C019F5000E1A6F8FEC10F009
:102ECC000001E12B300E0401685D006E0A0E000259
:102EDC00F3CF01F0300E695D006E0050012601C089
:102EEC003BF00101C151015C04E3BE513B5CD8A035
:102EFC00336A000E3B5C05E3C1513B5C02E2010E00
:102F0C00336EBE513B5C02E3010E336E3350010A4B
:102F1C000EE10A0E05012B6F2C6B2D6B2E6B2F6B9C
:102F2C00306B316B326B336B59EC02F015D0050101
:102F3C000A0E2B6F35C02CF535C02DF535C02EF58E
:102F4C0035C02FF535C030F535C031F535C032F50B
:102F5C0035C033F559EC02F0000E0201531902E1B1
:102F6C00010E5219D8A49CEF1EF08F0E0501176F9D
:102F7C00040E186F3AEC09F077EC06F08F0E050191
:102F8C00176F040E186F360E196F000E1A6F3CEC8B
:102F9C000CF000C054F201C055F2000E026E01504C
:102FAC00025C02E1005000083AE28F0E0501216F2D
:102FBC00040E226FF8EC06F000C0E4F001C0E5F05E
:102FCC00800E026E800E0118025C02E100500608B1
:102FDC001EE2800E0001E519006E800E005C02E11D
:102FEC00540EE45D14E2440E0501176F000E186FC9
:102FFC003AEC09F0E6C017F5E7C018F5930E196F17
:10300C00040E1A6F7DEC0CF00101C08105D0E6C0F6
:10301C00E1FFE7C0E2FFE66A0201546B556B8F0ECD
:10302C000501176F040E186F3C0E196F000E1A6F06
:10303C003CEC0CF000C054F201C055F2000E026ED4
:10304C000150025C02E10050000818E20101BF8B44
:10305C008F0E0501216F040E226FF8EC06F000C0F4
:10306C00E4F001C0E5F0320E216F4B0E226F000E22
:10307C00236FD9EC06F00201546B556B8F0E0501D2
:10308C00176F040E186F950E196F000E1A6F3CEC2B
:10309C000CF000C054F201C055F2000E026E01504B
:1030AC00025C02E1005000080EE20101BF9B890E98
:1030BC000501216F480E226F000E236FD9EC06F02C
:1030CC000201546B556B8F0E0501176F040E186FB0
:1030DC00B80E196F000E1A6F3CEC0CF000C054F2D5
:1030EC0001C055F2000E026E0150025C02E100506C
:1030FC000008D8B0EFD002013D6B3E6B060E542594
:10310C00E96E000E5521EA6EEECF2BF5AAEC02F01B
:10311C000052D8B4D3D0070E02015425E96E000E2C
:10312C005521EA6EEECF2BF5AAEC02F00052D8B482
:10313C00C5D0060E02015425E96E000E5521EA6E2B
:10314C00300EEE5C006E016A000E015A0A0E046E1F
:10315C00000E056EEEEC03F000C015F501C016F57F
:10316C0015C53DF216C53EF2070E5425E96E000E4C
:10317C005521EA6E300EEE5C006E016A000E015AAB
:10318C000A0E046E000E056ED4EC0CF008C000F0B4
:10319C0009C001F0005005011525026E01501621E1
:1031AC00036E02C03DF203C03EF2800E006E800E34
:1031BC000318005C02E10250050876E2800E020161
:1031CC003E19006E800E005C02E1640E3D5D6CE207
:1031DC00280E0501216F4C0E226F000E236FD9ECC7
:1031EC0006F094C017F5C40E0501186F010E196F87
:1031FC002BEC0FF0C40E176F010E186F3AEC09F0A0
:10320C0077EC06F002013D5164080001946F060E44
:10321C000501176F000E186F060E02015425E96E9A
:10322C00000E5521EA6EEECF19F591EC0EF0030E5F
:10323C000B6E080E0C6E770E0D6E0D2EFED70C2E2F
:10324C00FCD70B2EFAD7070E0501176F000E186F5F
:10325C00070E02015425E96E000E5521EA6EEECFE1
:10326C0019F591EC0EF0030E0B6E080E0C6E770E2A
:10327C000D6E0D2EFED70C2EFCD70B2EFAD71D0E75
:10328C000501216F4D0E226F000E236FD9EC06F055
:10329C000501176B186BC40E196F010E1A6FC9EC70
:1032AC0009F077EC06F009D0D80E0501216F490E14
:1032BC00226F000E236FD9EC06F009D0410E0501E8
:1032CC00216F4A0E226F000E236FD9EC06F002011B
:1032DC00546B556B8F0E0501176F040E186FC70ECC
:1032EC00196F000E1A6F3CEC0CF000C054F201C0C8
:1032FC0055F2000E026E0150025C02E10050000813
:10330C00D8B0EED002013D6B3E6B040E5425E96E35
:10331C00000E5521EA6EEECF2BF5AAEC02F000520E
:10332C00D8B4D2D0050E02015425E96E000E5521F9
:10333C00EA6EEECF2BF5AAEC02F00052D8B4C4D052
:10334C00040E02015425E96E000E5521EA6E300E72
:10335C00EE5C006E016A000E015A0A0E046E000E3D
:10336C00056EEEEC03F000C015F501C016F515C5A1
:10337C003DF216C53EF2050E5425E96E000E5521A0
:10338C00EA6E300EEE5C006E016A000E015A0A0EF7
:10339C00046E000E056ED4EC0CF008C000F009C0F1
:1033AC0001F0005005011525026E01501621036E27
:1033BC0002C03DF203C03EF2800E006E800E031878
:1033CC00005C02E10250000875E2800E02013E1919
:1033DC00006E800E005C02E10B0E3D5D6BE2500E48
:1033EC000501216F4C0E226F000E236FD9EC06F0F5
:1033FC0060C017F5C40E0501186F010E196F2BEC88
:10340C000FF0C40E176F010E186F3AEC09F077EC41
:10341C0006F03DC260F0140E0501176F000E186F18
:10342C00040E02015425E96E000E5521EA6EEECF12
:10343C0019F591EC0EF0030E0B6E080E0C6E770E58
:10344C000D6E0D2EFED70C2EFCD70B2EFAD7150EAB
:10345C000501176F000E186F050E02015425E96E59
:10346C00000E5521EA6EEECF19F591EC0EF0030E1D
:10347C000B6E080E0C6E770E0D6E0D2EFED70C2EED
:10348C00FCD70B2EFAD7350E0501216F4D0E226F8E
:10349C00000E236FD9EC06F0100E0501176F000E0D
:1034AC00186FC40E196F010E1A6FC9EC09F077EC86
:1034BC0006F009D01F0E0501216F4A0E226F000E77
:1034CC00236FD9EC06F009D0840E0501216F4A0E4A
:1034DC00226F000E236FD9EC06F00201546B556B72
:1034EC008F0E0501176F040E186FBF0E196F000EAB
:1034FC001A6F3CEC0CF000C054F201C055F2000EF7
:10350C00026E0150025C02E100500008D8B078D085
:10351C0002013D6B3E6B070E5425E96E000E5521E2
:10352C00EA6EEECF2BF5AAEC02F0005266E0070E25
:10353C0002015425E96E000E5521EA6E300EEE5C48
:10354C00016E026A000E025A01C03DF202C03EF248
:10355C00800E006E800E0218005C02E10150000823
:10356C0043E2800E3E19006E800E005C02E1070EF5
:10357C003D5D3AE2050E006E3DC2E4F03EC2E5F060
:10358C00005006E00001E437E491E537FF0FF9D76E
:10359C000001200EE427000EE523600E0501216FCB
:1035AC004B0E226F000E236FD9EC06F0E4C017F51A
:1035BC00E5C018F5C40E0501196F010E1A6FB2ECB7
:1035CC000EF0C40E176F010E186F3AEC09F077EC81
:1035DC0006F0E6C017F5E7C018F5E4C019F5E5C02C
:1035EC001AF538EC0DF009D00501280E216F480EA4
:1035FC00226F000E236FD9EC06F00201546B556B51
:10360C0004018F51550A2FE1A2513B0A04E0A2514B
:10361C00230A01E028D077EC0DF0B30E0501216FE1
:10362C004B0E226F000E236FD9EC06F05A0E0501DB
:10363C00176F020E186F3AEC09F05C0E216F4C0EEE
:10364C00226F000E236FD9EC06F0680E0501176F80
:10365C00040E186F3AEC09F077EC06F004018F6B4E
:10366C000201546B556B8F0E0501176F040E186F0A
:10367C00A90E196F000E1A6F3CEC0CF000C054F23E
:10368C0001C055F2000E026E0150025C02E10050C6
:10369C00000876E20E0E0501216F460E226F000E19
:1036AC00236FD9EC06F0010E0101686F000E696FF3
:1036BC00800E6919006E800E005C02E1050E685DDB
:1036CC005CE2050E026E68C100F069C101F00250A7
:1036DC0005E0003600900136FF0FFAD700C0E4F089
:1036EC0001C0E5F0BAC117F5BBC118F500C019F55A
:1036FC0001C01AF538EC0DF0890E216F4C0E226FBB
:10370C00000E236FD9EC06F0E4C017F5E5C018F5F0
:10371C00C40E0501196F010E1A6FB2EC0EF0C40E37
:10372C00176F010E186F3AEC09F0090E3A6FB1ECF5
:10373C0000F0BAC117F5BBC118F53AEC09F077ECFB
:10374C0006F0BAC117F5BBC118F594C019F5000EF7
:10375C0005011A6F8FEC10F0520E0B6E2B0E0C6EC7
:10376C00000E0D6E0D2EFED70C2EFCD70B2EFAD79D
:10377C0000000101684B692B9BD70201546B556B00
:10378C008F0E0501176F040E186FA30E196F000E24
:10379C001A6F3CEC0CF000C054F201C055F2000E54
:1037AC00026E0150025C02E1005000083CE2A40EE3
:1037BC000501216F4A0E226F000E236FD9EC06F023
:1037CC006EEC0FF0490E216F4B0E226F000E236F23
:1037DC00D9EC06F072EC10F00A0E2B6F35C02CF5FC
:1037EC0035C02DF535C02EF535C02FF535C030F56B
:1037FC0035C031F53550010F006E00C032F500C0F8
:10380C0033F559EC02F0520E0B6E2B0E0C6E000EB3
:10381C000D6E0D2EFED70C2EFCD70B2EFAD70000FA
:10382C000201546B556B8F0E0501176F040E186F48
:10383C00B30E196F000E1A6F3CEC0CF000C054F272
:10384C0001C055F2000E026E0150025C02E1005004
:10385C0000080EE23E0E0501216F410E226F000E94
:10386C00236FD9EC06F077EC06F00201546B556B24
:10387C008F0E0501176F040E186FAE0E196F000E28
:10388C001A6F3CEC0CF000C054F201C055F2000E63
:10389C00026E0150025C02E100500008D8B0B4D0B6
:1038AC008F0E0501216F040E226FF8EC06F0000E4E
:1038BC00011802E1060E0018D8A4A6D0020E216F42
:1038CC004D0E226F000E236FD9EC06F0400E050151
:1038DC00176F000E186FBAC119F5BBC11AF5C9ECF8
:1038EC0009F077EC06F0020E0B6EA00E0C6E920E29
:1038FC000D6E0D2EFED70C2EFCD70B2EFAD700001A
:10390C00040E02015425E96E000E5521EA6EEECF2D
:10391C002BF5AAEC02F0005274E0050E02015425BE
:10392C00E96E000E5521EA6EEECF2BF5AAEC02F0F3
:10393C00005267E0040E02015425E96E000E552179
:10394C00EA6E300EEE5C566F0A0E5603F3CF00F0A3
:10395C00050E5425D96E000E5521DA6EDE50002668
:10396C00300E005C016E01C04FF20150010840E2C4
:10397C000F0E4F5D3DE2440E0501176F000E186FE0
:10398C00040E02015425E96E000E5521EA6EEECFAD
:10399C0019F591EC0EF0020E0B6EA00E0C6E920E41
:1039AC000D6E0D2EFED70C2EFCD70B2EFAD7000069
:1039BC00450E0501176F000E186F050E02015425F8
:1039CC00E96E000E5521EA6EEECF19F591EC0EF072
:1039DC00020E0B6EA00E0C6E920E0D6E0D2EFED7FF
:1039EC000C2EFCD70B2EFAD700004FC235F009D0A5
:1039FC00590E0501216F480E226F000E236FD9EC72
:103A0C0006F00201546B556B8F0E0501176F040EF7
:103A1C00186FCC0E196F000E1A6F3CEC0CF000C036
:103A2C0054F201C055F2000E026E0150025C02E12C
:103A3C0000500008D8B077D18F0E0501216F040E0D
:103A4C00226FF8EC06F0800E0118026E800E025CFC
:103A5C0002E1090E005CD8A066D1090E02015425C2
:103A6C00E16E000E5521E26EE66AF30E0501216F40
:103A7C004C0E226F000E236FD9EC06F0200E0501C0
:103A8C00176F000E186FC40E196F010E1A6FC9EC68
:103A9C0009F0040E02015425E96E000E5521EA6E60
:103AAC00EECF2BF5AAEC02F000C015F5050E0201C5
:103ABC005425E96E000E5521EA6EEECF2BF5AAECDB
:103ACC0002F000501527166B000E1623070E02018C
:103ADC005425E96E000E5521EA6EEECF2BF5AAECBB
:103AEC0002F000501527000E1623080E0201542573
:103AFC00E96E000E5521EA6EEECF2BF5AAEC02F022
:103B0C0000501527000E162315C550F216C551F29C
:103B1C00040E02015425E96E000E5521EA6E300E9A
:103B2C00EE5C006E016A000E015A0A0E046E000E65
:103B3C00056EEEEC03F0050E5425D96E000E5521E2
:103B4C00DA6EDE5000240001E46F000E0120E56FF8
:103B5C00300EE45F000EE55B070E02015425E96EA2
:103B6C00000E5521EA6E300EEE5C006E016A000EFE
:103B7C00015A0A0E046E000E056EEEEC03F0080EF0
:103B8C005425D96E000E5521DA6EDE5000243D6F9F
:103B9C00000E01203E6F300E3D5F000E3E5B000EAE
:103BAC000501161902E1040E1519D8A4AED0800E29
:103BBC000001E519006E800E005C02E10F0EE45D61
:103BCC00D8A0A3D0800EE519006E800E005C02E137
:103BDC00180EE45DD8B099D0800E006E800E0201F4
:103BEC003E19005C02E13D510308D8B08ED0800E26
:103BFC00006E800E3E19005C02E13D510B08D8A00E
:103C0C0084D0E4C0BEF1040E5425E96E000E55219B
:103C1C00EA6EEECF56F2240E0501176F000E186FE8
:103C2C0056C219F591EC0EF0050E02015425E96E01
:103C3C00000E5521EA6EEECF56F2250E0501176FD8
:103C4C00000E186F56C219F591EC0EF0030E0B6EA8
:103C5C00080E0C6E770E0D6E0D2EFED70C2EFCD7AB
:103C6C000B2EFAD73DC2C1F1070E02015425E96EA5
:103C7C00000E5521EA6EEECF56F2270E0501176F96
:103C8C00000E186F56C219F591EC0EF0030E0B6E68
:103C9C00080E0C6E770E0D6E0D2EFED70C2EFCD76B
:103CAC000B2EFAD7080E02015425E96E000E552191
:103CBC00EA6EEECF56F2280E0501176F000E186F44
:103CCC0056C219F591EC0EF0030E0B6E080E0C6E2D
:103CDC00770E0D6E0D2EFED70C2EFCD70B2EFAD7B1
:103CEC00EB0E0501216F4C0E226F000E236FD9ECE9
:103CFC0006F0200E0501176F000E186FC40E196F19
:103D0C00010E1A6FC9EC09F009D0500E0501216F94
:103D1C00470E226F000E236FD9EC06F077EC06F0FD
:103D2C000201546B556B0201546B556B2CEF15F063
:023D3C00FFD7AF
:104D480010EE19F0470E006E010E016EC70EF66EDA
:104D5800450EF76E000EF86E2DEC0AF010EE61F0BD
:104D6800060E006E010E016E230EF66E4D0EF76EE6
:104D7800000EF86E2DEC0AF010EE60F0010E006ED9
:104D8800010E016E060EF66E000EF76E000EF86E3E
:104D98002DEC0AF010EE67F0720E006E010E016E37
:104DA800460EF66E430EF76E000EF86E2DEC0AF006
:024DB8001200E7
:0100060004F5
:103D3E000000000000000000000000000000000075
:103D4E000000000000000000000000000000000065
:103D5E000000000000000000000000000000000055
:103D6E000000000000000000000000000000000045
:103D7E000000000000000000000000000000000035
:103D8E000000000000000000000000000000000025
:103D9E000000000000000000000000000000000015
:103DAE000000000000000000000000000000000005
:103DBE0000000000000000000000000000000000F5
:103DCE0000000000000000000000000000000000E5
:103DDE0000000000000000000000000000000000D5
:103DEE0000000000000000000000000000000000C5
:103DFE0000000000000000000000000000000000B5
:103E0E0000000000000000000000000000000000A4
:103E1E000000000000000000000000000000000094
:103E2E000000000000000000000000000000000084
:103E3E00000000000000000000005F000000000015
:103E4E000007000700000000147F147F140000001C
:103E5E00242A7F2A120000002616083432000000A1
:103E6E0076495522500000000000050300000000B6
:103E7E00001C2241000000000041221C0000000036
:103E8E0014083E081400000008083E080800000050
:103E9E00005030000000000008080808080000006C
:103EAE000060600000000000201008040200000006
:103EBE003E5149453E00000000427F400000000098
:103ECE0042615149460000002141454B310000003E
:103EDE001814127F100000002745454539000000D8
:103EEE003C4A4949300000000101790503000000F9
:103EFE003649494936000000064949291E0000008E
:103F0E0000363600000000000056360000000000AB
:103F1E0000081422410000001414141414000000B0
:103F2E0041221408000000000201510906000000A1
:103F3E003E4149555E0000007E1111117E000000C9
:103F4E007F494949360000003E41414122000000B0
:103F5E007F4141221C0000007F4949494100000079
:103F6E007F090909010000003E4149493A0000005D
:103F7E007F0808087F00000000417F41000000001C
:103F8E002041413F000000007F0814224100000044
:103F9E007F404040400000007F020C027F00000086
:103FAE007F0408107F0000003E4141413E000000AA
:103FBE007F090909060000003E4151215E00000004
:103FCE007F09192946000000464949493100000081
:103FDE0001017F01010000003F4040403F00000012
:103FEE001F2040201F0000003F403C403F000000CB
:103FFE00631408146300000007087008070000002F
:10400E006151494543000000007F4141000000001E
:10401E0002040810200000000041417F0000000053
:10402E000402010204000000404040404000000035
:10403E0000010204000000002054545478000000D7
:10404E007F484444380000003844444420000000B7
:10405E00384444487F00000038545454180000007F
:10406E00087E090102000000085454543C00000070
:10407E007F0804047800000000447D40000000002A
:10408E002040443D000000007F1028440000000046
:10409E0000417F40000000007C04180478000000FE
:1040AE007C080404780000003844444438000000C2
:1040BE007C14141408000000081414187C0000006E
:1040CE007C080404080000004854545420000000EA
:1040DE00043F4440200000003C4040207C00000093
:1040EE001C2040201C0000003C4038403C000000DA
:1040FE0044281028440000000C5050503C00000092
:10410E004464544C44000000000836410000000096
:10411E0000007F0000000000004136080000000093
:10412E000000060909060000001038541010100097
:10413E003C48656C703E202063657474652061692F
:10414E00646520210D0A3C4D73673D3E2020204CB6
:10415E00206D6178693D31323020636172730D0AD2
:10416E003C52657365743E202052652D496E69740C
:10417E002061666669636865757273204D415837B4
:10418E003231390D0A3C54454D505F4F4E3E202082
:10419E002041666669636865206C612054656D70A8
:1041AE002E20445331384232300D0A3C54454D5086
:1041BE005F4F46463E2020456E6C65766520416613
:1041CE006669636861676520445331384232300D49
:1041DE000A3C53706565643D33303E20202056699D
:1041EE00746573736520646566696C656D656E7460
:1041FE00203A76616C65757220646520303520E05A
:10420E002039380D0A3C4C756D3D30343E2020204F
:10421E00204C756D696E6F736974E9204D61786914
:10422E002020303220E0203134200D0A3C456570CC
:10423E00726F6D3D323E2020204D65737361676550
:10424E0020656E20656570726F6D20646520333257
:10425E002063617273202C6176656320696E6469D8
:10426E006365203120E020360D0A3C504C4D3D3127
:10427E00383A30363E20506C616765204C756D695A
:10428E006E6F736974E9204D696E696D616C65209E
:10429E000D0A3C5265703D30313E20202052657033
:1042AE0065746974696F6E204D65737361676520FF
:1042BE0020303120E02031300D0A3C553B30343B6C
:1042CE0030363B31393B32303B35393B30343B2392
:1042DE003E20206F75202E2E2E30343B233E204D57
:1042EE00616A206465206C612052544320553B4A1C
:1042FE004A3B4D4D3B41413B48483B4D4D3B4A535C
:10430E003B23200D0A3C44656D6F3E2020206166E4
:10431E00666963686520746F7573206C6573206DB4
:10432E006573736167657320656E20454550524F06
:08433E004D205049430D0A0017
:10434600E84800804400B843001C4400D64600FC00
:1043560049002F4500674900D9440053460053469B
:0D43660000F54700C44A00444D00B74C006C
:014373001E2B
:0943740054454D505F4F464600D0
:01437D00003F
:02437E0000003D
:0243800000003B
:0643820052657365740032
:0543880044656D6F00AB
:05438D004C756D3D00C0
:0543920048656C70009D
:0743970053706565643D00F1
:08439E00456570726F6D3D0072
:0543A6005265703D00AE
:0543AB00504C4D3D00E7
:0443B0000000000009
:0443B4000000000005
:1043B8002050726F6A6574203A20486F726C6F677C
:1043C800655F4D6573736167655F446566696C61B8
:1043D8006E745F38784D6178373231395F4D61746A
:1043E80072696365735F565F31384632366B3232B5
:1043F8005F466F73635F696E7465726E655F3634AE
:104408004D687A5F323032305F31322E6D637070B2
:04441800690D0A0020
:10441C0020536F75726365203A20486F726C6F671A
:10442C00655F4D6573736167655F446566696C6153
:10443C006E745F38784D6178373231395F4D617405
:10444C0072696365735F565F31384632366B323250
:10445C005F466F73635F496E7465726E655F363469
:10446C004D487A5F5F323032305F313232302E63FA
:04447C00200D0A0005
:10448000204469726563746F7279203A20433A5C04
:104490005F4D696B726F435C5F4D657350726F6AFD
:1044A0006574735F4D696B726F435C486F726C6FBC
:1044B00067655F6465665F385F6D617472696365C7
:1044C000735F566572746963616C65735F313846FA
:0944D00032364B3232200D0A0095
:1044D90020454550524F4D203A486F726C6F6765C1
:1044E9005F4D6573736167655F446566696C616E8D
:1044F900745F38784D6178373231395F4D61747244
:10450900696365735F565F31384632366B32325FA5
:10451900323032305F31305F454550524F4D2E6950
:064529006865780D0A0030
:10452F00205350493120536F667477202D3E204D14
:10453F004158373231392C204932433120485720E6
:10454F002D3E204453313330372C205541525431B6
:10455F0020313930302C382C4E2C312C204F5753E2
:0C456F002D3E445331384232300D0A001A
:10457B00204C756D696E6F736974E92043726F69B6
:10458B007373616E7465206465206C61206761755F
:10459B006368652076657273206C612064726F6945
:1045AB007465203A2031352C31332C31302C382C9A
:0C45BB00362C332C322C3020200D0A004E
:1045C700934C00294D00174D007F4C002F4D00A53F
:0845D7004C00104D00C04C0027
:0245DF000000DA
:0145E10000D9
:0145E20000D8
:0145E30004D3
:0545E4004D73673D006E
:0145E90000D1
:0845EA0054454D505F4F4E0097
:1045F2000D0A2068656C6C6F2C2069206765742039
:0C460200796F7572204D7367210D0A005E
:10460E00416666696368652036204D657373616720
:10461E00657320656E20454550524F4D206D6F6479
:10462E00756C6F20333220E02070617274697220D5
:10463E006465203078303034302E2E30783030456E
:05464E0030200D0A0000
:104653002038204D6174726963657320387838207F
:10466300726163636F7264656D656E7420766572E3
:10467300746963616C2048415554207665727320D8
:1046830042617320737572204D4158373132390DB1
:024693000A001B
:1046950020553A30333B31323B31393B31383B33AE
:1046A500363B3032232020706F7572203033206402
:1046B5006563656D6272652032303139202031388D
:1046C5004833362030323D4D617264690D0A0D0A5A
:0146D50000E4
:1046D60020436F6E666967204269747320503138D3
:1046E6004632364B32325F426173655F466F7363A3
:1046F6005F696E7465726E655F313678504C4C5FDB
:0F47060036344D487A2E6366677363680D0A0078
:10471500496E6974204932433120285243333D5351
:10472500434C206574205243343D53444120293184
:1047350030304B687A200D0A20496E697420525436
:0B47450043204453313330370D0A008D
:104750002042414420504C4D2076616C7565732198
:10476000206D7573742062652066726F6D205B31F9
:10477000352E2E203233205D20746F205B203420B4
:084780002E2E203131205D00D6
:10478800496E69742053504920536F66747761727B
:10479800652020524332202853434B292C20524372
:1047A80031202853444F2C2920657420524330204F
:0847B80028435329200D0A00DB
:1047C0000D0A2052617070656C20666F726D6174A5
:1047D00020646520636465203A2022553B4A4A3BA9
:1047E0004D4D3B41413B48483B4D4D3B6A533B237C
:0547F00022200D0A006B
:1047F5002053616973697220756E206E6F757665D9
:104805006175204D73672061766563206C65207442
:1048150065726D696E616C20766961204D73673DC7
:034825000D0A0079
:104828000D0A20456570726F6D204D7367206164B5
:10483800726573736520206D7573742062652077C7
:10484800697468696E203120746F20373E3E0D0A06
:01485800005F
:1048590020424144204E756D2076616C756520219A
:10486900206D75737420626520696E2074686520F7
:1048790072616E67652030322E2E3134200D0A00A8
:104889000D0A204F4B2C2054656D70657220697399
:10489900204F4646210D0A5265746F757220617565
:1048A90020646973706C617920747874200D0A0032
:1048B900204C756D696E6F736974E92052E92D6931
:1048C9006E697469616C6973E96520617665632055
:0F48D90076616C657572204C756D20200D0A009C
:1048E800204C616E6761676520204D696B726F634C
:1048F800205620372E36300D0A204D4355203A20B9
:0B49080031384632364B32320D0A00C7
:1049130020446973706C6179203C30313233343513
:1049230036373E207375722038206D617472696367
:0B4933006573204C656473200D0A00C2
:10493E0020415454454E54494F4E203A20496E69F9
:10494E0074204843303520E0203139323030206237
:09495E0061756473203A0D0A0032
:1049670020506F77657220537570706C7920352EE3
:104977003056202620332E387620666F72204D6100
:07498700747269780D0A004B
:10498E0020526563757020506172616D6574726539
:10499E007320656E2045656570726F6D20504943BA
:0549AE00203A0D0A0093
:1049B3000D0A20436C6F636B20696E697469616CC7
:1049C3006520696E20203D20202E2E2E20204B684E
:0549D3007A200D0A002E
:1049D8000D0A205370656564206D757374206265D7
:1049E8002077697468696E20303520746F203938F3
:0449F800200D0A0084
:1049FC0020464F5343203D464F534320496E746528
:104A0C00726E6520313678504C4C3D36344D487AB8
:034A1C000D0A0080
:104A1F000D0A20526570206D7573742062652077C2
:104A2F00697468696E20303120746F203130200D29
:024A3F000A006B
:104A41000D0A2042414420636465202C206D75735A
:104A5100742062653A2053706565643D7878200D55
:024A61000A0049
:104A63000D0A45727265757220737572204A6F75EF
:104A7300722053656D61696E65206A532E200D0A9D
:014A83000032
:104A84000D0A2042414420636465202C206D757317
:104A9400742062653A205265703D7878200D0A00D2
:104AA40052657365742041666669636865757273DF
:104AB400204D61747269636520387838200D0A00CE
:104AC400204D6F64652054656D70657261747572F4
:0F4AD4006520617665632054454D505F4F4E005D
:104AE3000D0A45637269747572652064616E732083
:0F4AF3004453313330372E2E2E204F4B0D0A00F7
:104B020020436C656172204D61747269636520385F
:084B120078203878380D0A0004
:104B1A00204C756D696E6F736974E9204D696E6911
:084B2A006D616C65200D0A00AD
:104B32000D0A204F4B2C2054656D706572206973ED
:074B4200204F4E210D0A0077
:104B4900436C656172204D617472696365203678C2
:074B5900203878380D0A0036
:104B60002020456570726F6D204D736720616472FF
:064B70006573736520006F
:104B760041542B4E414D453D484330355F34313825
:054B860030560D0A008D
:104B8B0054657374207265672E204453313842325A
:044B9B00300D0A00CF
:104B9F0041542B554152543D31393230302C302C49
:044BAF00300D0A00BB
:104BB3004E65772044533133303720446174652088
:024BC3003A00B6
:104BC5000A0D205254432055704461746564200DCC
:024BD5000A00D4
:104BD7002052652D4C6563747572652052544320CD
:014BE70000CD
:104BE80020506573656E746174696F6E203A0D0AA2
:014BF80000BC
:104BF900303132333435363738394142434445460A
:104C0900204453313330372044617465203A200001
:0F4C190046616D696C7920436F6465203A200015
:0E4C2800204F6C64207370656564203D200091
:0D4C360041542B50494E313233340D0A00E9
:0D4C430041542B56455253494F4E0D0A0067
:0C4C5000204F6C6420526570203D200055
:0C4C5C00204E65772054696D653A2000F9
:0C4C680041542B524E414D453F0D0A00B7
:0B4C740041542B554152543F0D0A00E3
:0A4C7F004D657263726564692E00D2
:0A4C8900456570726F6D2023200056
:094C930050726F626C656D6F00D8
:094C9C0030313233343536370073
:094CA50056656E647265646900D5
:094CAE00202020202020202000FD
:094CB700207878787878782000E4
:094CC00044696D616E63686500D2
:094CC900202020202020202000E2
:094CD200202020202020202000D9
:084CDB002054696D653A2000C8
:084CE30020204352433D200054
:084CEB00204E6577203D2000FA
:084CF300204F6C64203D2000FD
:074CFB00204944313D200077
:074D0200204C756D3D2000FF
:074D0900204370743D2000FF
:074D100053616D6564690049
:064D17004D6172646900A9
:064D1D00204E6577200026
:024D230000008E
:024D250020006C
:024D270020006A
:064D29004C756E64690088
:064D2F004A65756469008D
:064D3500204E657720000E
:054D3B0041540D0A00C7
:044D4000B04320005C
:044D4400202020000B
:020000040030CA
:0D00010038183CFFBF81FF0FC00FE00F401B
:0200000400F00A
:1000000053706565643D333000FFFFFFFFFFFFFF66
:100010005265703D303400FFFFFFFFFFFFFFFFFF21
:10002000504C4D3D31393A303500FFFFFFFFFFFFA7
:10003000416E4E6575663D323100FFFFFFFFFFFFE9
:100040004C756D3D303200FFFFFFFFFFFFFFFFFFEC
:1000500020313846323538204D696B726F204300AD
:1000600032656D20436F75636F752000FFFFFFFFE2
:10007000FFFFFFFFFFFFFFFFFFFFFFFFFFFFFFFF90
:1000800033656D20204F756920204F4B204241443D
:1000900000FFFFFFFFFFFFFFFFFFFFFFFFFFFFFF6F
:1000A00034656D206D6573736167652020202020A5
:1000B0002020202020202020202020202020200060
:1000C00035656D204D73672E2E2E2E2E2E2E2E2E44
:1000D0002E2E2E2E2E2E2E2E2E2E2E2E2E2E2E006E
:1000E00036656D204D657373616765202020202083
:1000F0002E2E2E2E2E2E2E2E2E2E2E2E2E2E2E004E
:10010000FFFFFFFFFFFFFFFFFFFFFFFFFFFFFFFFFF
:10011000FFFFFFFFFFFFFFFFFFFFFFFFFFFFFFFFEF
:10012000FFFFFFFFFFFFFFFFFFFFFFFFFFFFFFFFDF
:10013000FFFFFFFFFFFFFFFFFFFFFFFFFFFFFFFFCF
:00000001FF
